:020000040000FA
:020000000528D1
:0800080009008316FF2390009C
:1000100007309500003081002030960083120030B8
:100020008B00073099000030850010308700A60152
:1000300083160F3085000F3087008312A801A901B5
:10004000D830AA00A80A031D2B28A90A031D2B28B3
:10005000AA0A03193228D92000002108FF3A031DFB
:100060004828222883168516831205160712831640
:100070002830850000308700831210308500003062
:10008000870008308B00851A630000008B0113285D
:10009000E220E220E220E220E220F320FA20F32016
:1000A000FA20F320FA20E220F32021185B28A60A88
:1000B000000000005E28FD20F320FA20E220F3205B
:1000C000A1186628A60A000000006928FD20F32078
:1000D000FA20E220F320211A7128A60A000000006D
:1000E0007428FD20F320FA20E220F320A11A7C28B6
:1000F000A60A000000007F28FD20F320FA20E2205D
:10010000F320211B8728A60A000000008A28FD2072
:10011000F320FA20E220F320A11B9028A60A9328BE
:10012000FD20F320FC202608A700E220F32027185A
:100130009D28A60A00000000A028FD20F320FA2038
:10014000E220F320A718A828A60A00000000AB2888
:10015000FD20F320FA20E220F3202119B328FC200F
:10016000E220F320B728FD20F320A60A0000A11901
:10017000BE28000000000000E220BF28A60A1030C0
:10018000A607F320FD20A60BC1282108A300643098
:10019000A4002B30A500D92021082306031D4828E0
:1001A000FF30210603191E28A50BCB28A40BC92854
:1001B000482805080F39A10007080F39A200220EB0
:1001C000A10400340B30A0008716F9208712F92013
:1001D000FC20A00BE42800008716F9208712F920E4
:1001E0000000000008004B30A0000000A00BF52824
:0C01F000080000000000000000000800F3
:02400E00043E6E
:00000001FF
